:100000000C9462000C948A000C948A000C948A0070
:100010000C948A000C948A000C948A000C948A0038
:100020000C948A000C948A000C948A000C948A0028
:100030000C948A000C948A000C948A000C948A0018
:100040000C9446020C948A000C94B6020C94900214
:100050000C948A000C948A000C948A000C948A00F8
:100060000C948A000C948A000000000025002800EF
:100070002B0000000000240027002A0000000000E0
:1000800023002600290004040404040404040202DA
:100090000202020203030303030301020408102007
:1000A0004080010204081020010204081020000012
:1000B0000008000201000003040700000000000027
:1000C0000000E80211241FBECFEFD8E0DEBFCDBF95
:1000D00011E0A0E0B1E0E8E9F3E102C005900D9283
:1000E000A033B107D9F721E0A0E3B1E001C01D9230
:1000F000A33FB207E1F710E0C2E6D0E004C02197C9
:10010000FE010E94C409C136D107C9F70E942D0320
:100110000C94CA090C940000833081F028F48130DB
:1001200099F08230A9F008958730A9F08830C9F09D
:100130008430B1F4809180008F7D03C08091800075
:100140008F7780938000089584B58F7784BD08955C
:1001500084B58F7DFBCF8091B0008F778093B00006
:1001600008958091B0008F7DF9CFCF93DF93282F32
:1001700030E0F901E255FF4F8491F901E656FF4F57
:10018000D491F901EA57FF4FC491CC23A1F081111A
:100190000E948C00EC2FF0E0EE0FFF1FE458FF4FA1
:1001A000A591B491EC91ED2381E090E009F480E019
:1001B000DF91CF91089580E090E0FACFCF93DF9365
:1001C00090E0FC01E656FF4F24918A579F4FFC01B7
:1001D00084918823C9F090E0880F991FFC01EE58A4
:1001E000FF4FA591B491FC01E859FF4FC591D491FF
:1001F00061110DC09FB7F8948C91209582238C9348
:100200008881282328839FBFDF91CF910895623092
:1002100051F49FB7F8943C91822F809583238C935F
:10022000E8812E2BEFCF8FB7F894EC912E2B2C93E7
:100230008FBFEACF8E50806480937C0080917A00DB
:10024000806480937A0080917A0086FDFCCF809153
:100250007800909179000895AF92BF92CF92DF928B
:10026000EF92FF920F931F93CF93DF936C017B016B
:100270008B01040F151FEB015E01AE18BF08C017FC
:10028000D10759F06991D601ED91FC910190F0816F
:10029000E02DC6010995892B79F7C501DF91CF9132
:1002A0001F910F91FF90EF90DF90CF90BF90AF9094
:1002B0000895FC01538D448D252F30E0842F90E06C
:1002C000821B930B541710F0CF9608950197089551
:1002D000FC01918D828D981761F0A28DAE0FBF2F1A
:1002E000B11D5D968C91928D9F5F9F73928F90E070
:1002F00008958FEF9FEF0895FC01918D828D9817DF
:1003000031F0828DE80FF11D858D90E008958FEF1B
:100310009FEF0895FC01918D228D892F90E0805CE4
:100320009F4F821B91098F739927089587E491E06D
:100330000E948A0121E0892B09F420E0822F089590
:1003400080E090E0892B29F00E94960181110C94A5
:1003500000000895FC01A48DA80FB92FB11DA35A68
:10036000BF4F2C91848D90E001968F739927848FD5
:10037000A689B7892C93A089B1898C9183708064F8
:100380008C93938D848D981306C00288F389E02D99
:1003900080818F7D80830895EF92FF920F931F934A
:1003A000CF93DF93EC0181E0888F9B8D8C8D981328
:1003B0001AC0E889F989808185FF15C09FB7F89434
:1003C000EE89FF896083E889F98980818370806480
:1003D00080839FBF81E090E0DF91CF911F910F91CB
:1003E000FF90EF900895F62E0B8D10E00F5F1F4FDA
:1003F0000F731127E02E8C8D8E110CC00FB607FCE9
:10040000FACFE889F989808185FFF5CFCE010E9476
:10041000AA01F1CFEB8DEC0FFD2FF11DE35AFF4F39
:10042000F0829FB7F8940B8FEA89FB898081806204
:10043000CFCFCF93DF93EC01888D8823B9F0AA89C1
:10044000BB89E889F9898C9185FD03C0808186FD8F
:100450000DC00FB607FCF7CF8C9185FFF2CF8081DE
:1004600085FFEDCFCE010E94AA01E9CFDF91CF91A8
:100470000895FC0101900020E9F73197AF01481B76
:10048000590BBC0187E491E00C942C011F920F9250
:100490000FB60F9211242F933F938F939F93AF9397
:1004A000BF938091430190914401A0914501B09187
:1004B00046013091420123E0230F2D3758F5019674
:1004C000A11DB11D209342018093430190934401EB
:1004D000A0934501B093460180913E0190913F0168
:1004E000A0914001B09141010196A11DB11D8093E1
:1004F0003E0190933F01A0934001B0934101BF9111
:10050000AF919F918F913F912F910F900FBE0F90C0
:100510001F90189526E8230F0296A11DB11DD2CF7A
:100520001F920F920FB60F9211242F933F934F9368
:100530005F936F937F938F939F93AF93BF93EF934B
:10054000FF9387E491E00E94AA01FF91EF91BF9190
:10055000AF919F918F917F916F915F914F913F915B
:100560002F910F900FBE0F901F9018951F920F9212
:100570000FB60F9211242F938F939F93EF93FF93B6
:10058000E0915701F09158018081E0915D01F09177
:100590005E0182FD1BC09081809160018F5F8F732F
:1005A00020916101821741F0E0916001F0E0E95B88
:1005B000FE4F958F80936001FF91EF919F918F91F6
:1005C0002F910F900FBE0F901F9018958081F4CF40
:1005D000E7E4F1E01382128288EE93E0A0E0B0E05D
:1005E00084839583A683B7838CE091E09183808395
:1005F00085EC90E09587848784EC90E097878687E8
:1006000080EC90E0918B808B81EC90E0938B828BDF
:1006100082EC90E0958B848B86EC90E0978B868BB8
:10062000118E128E138E148EE7EEF1E082E390E0CD
:10063000A0E0B0E080839183A283B383148215820B
:100640001682178281E08087818712861386E4EE06
:10065000F1E01082118212820895CF93DF93CDB71B
:10066000DEB760970FB6F894DEBF0FBECDBF7894AB
:1006700084B5826084BD84B5816084BD85B58260A7
:1006800085BD85B5816085BD80916E008160809358
:100690006E001092810080918100826080938100C1
:1006A00080918100816080938100809180008160D1
:1006B000809380008091B10084608093B10080912C
:1006C000B00081608093B00080917A008460809354
:1006D0007A0080917A00826080937A0080917A001B
:1006E000816080937A0080917A00806880937A009C
:1006F0001092C100E0915701F091580112E010836F
:10070000E0915301F09154011082E0915501F09174
:1007100056018FEC808310925F01E0915B01F091B4
:100720005C0186E08083E0915901F0915A0180815B
:1007300080618083E0915901F0915A018081886045
:100740008083E0915901F0915A0180818068808313
:10075000E0915901F0915A0180818F7D808360E0A2
:100760008EE00E94DE0060E08FE00E94DE0060E02C
:1007700080E10E94DE0061E083E00E94DE0062E032
:1007800084E00E94DE0060E081E10E94DE0061E022
:1007900089E00E94DE0061E08AE00E94DE0061E004
:1007A0008BE00E94DE0081EA8093800089E08093E4
:1007B000810083E88093B0001093B10000E810E05E
:1007C000109389000093880010938B0000938A0097
:1007D00080E88093B3008FB7F894C0904301D09025
:1007E0004401E0904501F09046018FBF84E00E94F3
:1007F000B5001092F1011092F2019091F001891769
:1008000051F08093F001C092EB01D092EC01E092A4
:10081000ED01F092EE018091EB019091EC01A0913D
:10082000ED01B091EE01C81AD90AEA0AFB0A8091DB
:10083000E7019091E801A091E901B091EA018C15DE
:100840009D05AE05BF05B0F49091EF018091F001D8
:10085000981781F08093EF01911103C021E081305E
:1008600009F020E02093F101913009F4811190E02A
:100870009093F2018091F2018823D1F060913D01C3
:1008800081E0682760933D0190E080E00E940E07C0
:1008900081E291E00E94390280913D018111C0C046
:1008A0008AE191E00E9439028DE291E00E943902D2
:1008B00081E10E94B5002091E401211103C091E083
:1008C000813009F090E09093E501213009F4811125
:1008D00020E02093E6018093E4019923E1F08DEC80
:1008E0009CECACECBDE38093040190930501A093D4
:1008F0000601B09307011092390110923A0110924B
:100900003B0110923C011092350110923601109279
:1009100037011092380100913D01098334E1C32E63
:10092000D12CE12CF12C45E0842E912CA12CB12C62
:10093000002349F09AE0C92ED12CE12CF12C812C16
:10094000912C540183948EE00E941A01A701960114
:10095000281939094A095B09DC010E9446072FEF73
:1009600033E040E050E00E941C07CA01B901680D65
:10097000791D8A1D9B1D0E949B082B013C018FE065
:100980000E941A012EE130E0DC010E94BD092FEF28
:1009900033E040E050E00E941C07CA01B9016C5EE0
:1009A0007F4F8F4F9F4F0E949B084B015C0180E15E
:1009B0000E941A0123E030E0DC010E94BD092FEF04
:1009C00033E040E050E00E941C07CA01B9016F5FAC
:1009D0007F4F8F4F9F4F0E949B086D877E878F8729
:1009E000988B8EE00E941A01853511E091070CF476
:1009F00009C28A3A9240BCF009818AE097EDA3E2ED
:100A0000BCE3011106C21AC01A821982F6C00FEFA8
:100A100010E01A830983F1C019811E2B1C93DCC1DD
:100A20008EE191E03FCF09818AE097EDA3EABBE335
:100A3000002321F08FE692E1A3E0BAE38093000166
:100A400090930101A0930201B093030180913901B9
:100A500090913A01A0913B01B0913C0189839A8326
:100A6000AB83BC83C0900401D0900501E0900601E7
:100A7000F090070100913501109136012091370166
:100A8000309138010D831E832F83388780910001B8
:100A900090910101A0910201B091030189879A8789
:100AA000AB87BC87A701960169817A818B819C8184
:100AB0000E947F07A30192010E94500929853A856F
:100AC0004B855C850E945009A70196010E94800712
:100AD0002B013C01409204015092050160920601F5
:100AE000709207012D813E814F815885C501B40167
:100AF0000E947F07A70196010E94500929813A812F
:100B00004B815C810E947F0729853A854B855C85F6
:100B10000E94500929813A814B815C810E948007A3
:100B20004B015C018092390190923A01A0923B0105
:100B3000B0923C01A701960169817A818B819C81E9
:100B40000E9450096B017C012D813E814F815885A7
:100B50006D857E858F8598890E9450099B01AC0127
:100B6000C701B6010E947F0729853A854B855C85C0
:100B70000E9450092D813E814F8158850E94800737
:100B80006B017C01C0923501D0923601E0923701B1
:100B9000F092380120E030E040EF51E4C301B201AF
:100BA0000E94800720E030E04FE753E40E945009A4
:100BB00020E030E040E752E40E94F10720E030E01E
:100BC000A9010E9480072B013C0120E030E0A9012F
:100BD0000E94EC0787FD18CF20E030E04FE753E498
:100BE000C301B2010E944B0918160CF410CFC301C7
:100BF000B2010E9463087A83698320E030E040EF0D
:100C000051E4C501B4010E94800720E030E04FE7C5
:100C100053E40E94500920E030E040E752E40E9493
:100C2000F10720E030E0A9010E9480074B015C0140
:100C300020E030E0A9010E94EC0710E000E087FD11
:100C400011C020E030E04FE753E4C501B4010E9439
:100C50004B090FEF10E018162CF0C501B4010E94EB
:100C600063088B0120E030E04FE753E4C701B60191
:100C70000E94500920E030E048E452E40E94F1076D
:100C800020E030E0A9010E9480076B017C0120E098
:100C900030E0A9010E94EC0760E087FD0FC020E072
:100CA00030E04FE753E4C701B6010E944B096FEFF4
:100CB000181624F0C701B6010E94630829813A8101
:100CC000309389002093880010938B0000938A0052
:100CD0006093B30020E034E244E759E460910001FE
:100CE0007091010180910201909103010E945009CD
:100CF0000E9463089B01AC0122533109410951094B
:100D0000AEE3BEEF0E9449072EED36E240E050E030
:100D10000E941C07BA01A9014C505E4F6F4F7F4FD4
:100D2000453F31E053076105710520F044EF51E084
:100D300060E070E0423351056105710520F442E343
:100D400050E060E070E08FB7F894C0904301D0901D
:100D50004401E0904501F09046018FBF8091310140
:100D600090913201A0913301B09134019701860135
:100D7000081B190B2A0B3B0BD901C801481759074F
:100D80006A077B0708F031C01091300181E0182715
:100D90001D8310933001E1EBF0E08491EDE9F0E088
:100DA00004910983E9E8F0E014911123B1F0811175
:100DB0000E948C00E12FF0E0EE0FFF1FE859FF4F7B
:100DC000A591B4918FB7F8941D81EC91111124CEA7
:100DD000098100950E230C938FBFC0923101D092F0
:100DE0003201E0923301F092340180E090E0892BEF
:100DF00009F4F1CC0E949601882309F4ECCC0E94FE
:100E00000000E9CC198187E197EBA1EDB8E311115E
:100E100015CE8FE692E1A3E8BAE310CE262FF9991A
:100E2000FECF1FBA92BD81BD20BD0FB6F894FA9ACD
:100E3000F99A0FBE01960895052E97FB1EF40094B3
:100E40000E94330757FD07D00E944E0707FC03D0CE
:100E50004EF40C94330750954095309521953F4FB3
:100E60004F4F5F4F089590958095709561957F4F96
:100E70008F4F9F4F08950E947007A59F900DB49FBC
:100E8000900DA49F800D911D11240895B7FF0C941F
:100E90003B070E943B07821B930B0895A1E21A2E89
:100EA000AA1BBB1BFD010DC0AA1FBB1FEE1FFF1F0E
:100EB000A217B307E407F50720F0A21BB30BE40B5E
:100EC000F50B661F771F881F991F1A9469F76095A5
:100ED0007095809590959B01AC01BD01CF0108955F
:100EE000A29FB001B39FC001A39F700D811D11246B
:100EF000911DB29F700D811D1124911D08955058B0
:100F0000BB27AA270E9497070C9411090E94030986
:100F100038F00E940A0920F039F49F3F19F426F4B2
:100F20000C9400090EF4E095E7FB0C94FA08E92F05
:100F30000E94220958F3BA176207730784079507BE
:100F400020F079F4A6F50C9444090EF4E0950B2EEC
:100F5000BA2FA02D0B01B90190010C01CA01A0010B
:100F60001124FF27591B99F0593F50F4503E68F166
:100F70001A16F040A22F232F342F4427585FF3CFA7
:100F8000469537952795A795F0405395C9F77EF478
:100F90001F16BA0B620B730B840BBAF09150A1F0C1
:100FA000FF0FBB1F661F771F881FC2F70EC0BA0F47
:100FB000621F731F841F48F4879577956795B795CF
:100FC000F7959E3F08F0B0CF9395880F08F09927CA
:100FD000EE0F9795879508950E94D60808F481E052
:100FE00008950E9405080C9411090E940A0958F0FE
:100FF0000E94030940F029F45F3F29F00C94FA089D
:1010000051110C9445090C9400090E94220968F3BF
:101010009923B1F3552391F3951B550BBB27AA27B1
:1010200062177307840738F09F5F5F4F220F331FEB
:10103000441FAA1FA9F335D00E2E3AF0E0E832D0B3
:1010400091505040E695001CCAF72BD0FE2F29D0B6
:10105000660F771F881FBB1F261737074807AB0788
:10106000B0E809F0BB0B802DBF01FF2793585F4FFD
:101070003AF09E3F510578F00C94FA080C9445091B
:101080005F3FE4F3983ED4F3869577956795B795DF
:10109000F7959F5FC9F7880F911D9695879597F9EA
:1010A0000895E1E0660F771F881FBB1F6217730763
:1010B0008407BA0720F0621B730B840BBA0BEE1F78
:1010C00088F7E09508950E946A086894B1110C941D
:1010D000450908950E942A0988F09F5798F0B92F72
:1010E0009927B751B0F0E1F0660F771F881F991F5D
:1010F0001AF0BA95C9F714C0B13091F00E944409B2
:10110000B1E008950C944409672F782F8827B85FC1
:1011100039F0B93FCCF3869577956795B395D9F7B4
:101120003EF490958095709561957F4F8F4F9F4FBE
:101130000895E89409C097FB3EF4909580957095CA
:1011400061957F4F8F4F9F4F9923A9F0F92F96E913
:10115000BB279395F695879577956795B795F11188
:10116000F8CFFAF4BB0F11F460FF1BC06F5F7F4F25
:101170008F4F9F4F16C0882311F096E911C0772337
:1011800021F09EE8872F762F05C0662371F096E840
:10119000862F70E060E02AF09A95660F771F881F0F
:1011A000DAF7880F9695879597F90895990F0008B3
:1011B000550FAA0BE0E8FEEF16161706E807F90729
:1011C000C0F012161306E407F50798F0621B730BC4
:1011D000840B950B39F40A2661F0232B242B252B45
:1011E00021F408950A2609F4A140A6958FEF811DE8
:1011F000811D089597F99F6780E870E060E0089589
:101200009FEF80EC089500240A941616170618061E
:101210000906089500240A941216130614060506FA
:101220000895092E0394000C11F4882352F0BB0F8B
:1012300040F4BF2B11F460FF04C06F5F7F4F8F4FEE
:101240009F4F089557FD9058440F551F59F05F3F29
:1012500071F04795880F97FB991F61F09F3F79F0D8
:1012600087950895121613061406551FF2CF46955A
:10127000F1DF08C0161617061806991FF1CF8695DC
:101280007105610508940895E894BB2766277727C0
:10129000CB0197F908950E94D60808F48FEF0895BE
:1012A0000E9463090C9411090E94030938F00E94FE
:1012B0000A0920F0952311F00C94FA080C94000907
:1012C00011240C9445090E94220970F3959FC1F3E3
:1012D000950F50E0551F629FF001729FBB27F00DE4
:1012E000B11D639FAA27F00DB11DAA1F649F662739
:1012F000B00DA11D661F829F2227B00DA11D621F88
:10130000739FB00DA11D621F839FA00D611D221F41
:10131000749F3327A00D611D231F849F600D211D25
:10132000822F762F6A2F11249F5750409AF0F1F0A8
:1013300088234AF0EE0FFF1FBB1F661F771F881F11
:1013400091505040A9F79E3F510580F00C94FA0847
:101350000C9445095F3FE4F3983ED4F38695779566
:101360006795B795F795E7959F5FC1F7FE2B880FB7
:10137000911D9695879597F908950E947007B7FF7C
:101380000895821B930B0895EE0FFF1F0590F491B3
:08139000E02D0994F894FFCF51
:101398000AD7233CCDCCCC3D00000000CC012C0169
:1013A800590119028A0168017C014F4646004F4ED7
:1013B80000536C6F77206D6F64653A20000D0A004A
:00000001FF
